:1000000012C02CC02BC02AC029C028C027C026C0BF
:1000100025C03BC123C02AC021C020C01FC01EC0B4
:100020001DC01CC01BC011241FBECFE5D4E0DEBF25
:10003000CDBF10E0A0E6B0E0ECEFF5E002C0059027
:100040000D92A038B107D9F710E0A0E8B0E001C0E8
:100050001D92AE38B107E1F75ED0CEC2D1CF10927B
:100060008000109281001092820008951F920F92DA
:100070000FB60F9211248F93EF93FF938CB180935F
:100080008300809182008830B8F4E0918000F0E035
:100090008CB1EA57FF4F8083809182008F5F8093FD
:1000A0008200809180008F5F80938000809180002B
:1000B000883011F410928000FF91EF918F910F9092
:1000C0000FBE0F901F90189580918200882311F425
:1000D000E0E016C0E0918100F0E0EA57FF4FE081D8
:1000E00080918200815080938200809181008F5F97
:1000F0008093810080918100883011F410928100FA
:100100008E2F08955D9BFECF8CB90895809183005A
:100110001092830008957F928F929F92AF92BF9228
:10012000CF92DF92EF92FF920F931F93DF93CF93C3
:1001300000D000D0CDB7DEB7B89AC09883B785603D
:1001400083BF89B7816089BF12BE68D1CAD181E0FF
:10015000BCD180EA9FE00197F1F710BC83E389B935
:1001600088E98AB986E880BD7894CC24DD24E6E964
:10017000EE2EF12CBB2470E5772E68EC862E912CA8
:1001800055E5A52E74D1082F88E89FD180E690E030
:10019000D8D1C7019DD0033019F48AE090E004C0A3
:1001A000043021F486EF9FEFE80EF91EEC14FD04F5
:1001B00030F4C09A88EC89D185E690E005C0C098FB
:1001C00088EC83D18EE690E0BCD1013039F491E027
:1001D000B91609F056C000E0BB2402C0BB20B1F440
:1001E0005D9BFECF7CB870DF182F109280001092BC
:1001F00081001092820080EC68D1812F8D52F7D05F
:1002000087E790E09ED181E0B81629F480EC5DD1BB
:100210008AE790E096D188EE93E0F4013197F1F708
:100220000197D9F7023029F55D9BFECFACB88091DC
:10023000860090E09A8389838091870090E09C8378
:100240008B831092800010928100109282008B812B
:100250009C8129813A81D82ECC24C20ED31E80E8FD
:1002600034D1C60135D080E236D18DE634D18DE669
:1002700032D188EE93E0F4013197F1F70197D9F785
:1002800081CF00E0BB24B394C1CF1F920F920FB671
:100290000F9211242F933F934F935F936F937F930C
:1002A0008F939F93AF93BF93EF93FF93BED0FF9134
:1002B000EF91BF91AF919F918F917F916F915F91DE
:1002C0004F913F912F910F900FBE0F901F90189557
:1002D000EF92FF920F931F939C0168EE73E078D129
:1002E000182F092FC90168EE73E072D1662311F44B
:1002F00080E302C0862F805DEED0812F902F64E6D0
:1003000070E066D1F82EE92E812F902F64E670E020
:100310005FD1662311F480E302C0862F805DDBD0BD
:100320008F2D9E2D6AE070E053D1362F8F2D9E2D9C
:100330006AE070E04DD1182F332311F480E302C03E
:10034000832F805DC8D0812F805DC5D01F910F9114
:10035000FF90EF9008950F931F939C0164E670E067
:1003600037D1182F092FC90164E670E031D1662317
:1003700011F480E302C0862F805DADD0812F902FD5
:100380006AE070E025D1362F812F902F6AE070E06F
:100390001FD1182F332311F480E302C0832F805D17
:1003A0009AD0812F805D97D01F910F9108951F9350
:1003B000282F64E601D1192F822FFED0882311F453
:1003C00080E301C0805D87D0812F6AE0F5D0282FBF
:1003D000812FF2D0192F222311F480E302C0822F43
:1003E000805D79D0812F805D76D01F9108951F9315
:1003F000282F6AE0E1D0382F822FDED0192F332347
:1004000011F480E302C0832F805D65D0812F805D71
:1004100062D01F910895805D5ED0089584B3807F7F
:1004200084BB85B38F6085BB0895989902C091E025
:100430000BC09A9902C093E007C0999902C092E05C
:1004400003C09B9911C094E080918500873420F00F
:100450008EE38093850005C08F5F80938500843094
:1004600029F4909384000895109285000895809156
:1004700084001092840008958093840008959AE681
:100480009A95F1F7C39892B3807F9F70982B92BB97
:10049000C19A85E08A95F1F7C198089592B3282F03
:1004A000207F9F70292B22BBC19A25E0922F9A951D
:1004B000F1F7C19892B38295807F9F70982B92BB81
:1004C000C19A2A95F1F7C19808959AE69A95F1F79D
:1004D000C398E4DF08959AE69A95F1F7C39ADEDFB0
:1004E00008950F931F9381B3806F81BBBB9ABA9A13
:1004F000B99A80E991E028EC30E0F9013197F1F701
:100500000197D9F780E3BBDF80E29EE40197F1F722
:1005100080E3B5DF00EA1FE0C8010197F1F780E34F
:10052000AEDF88E2ACDF88E2D0DF8CE0CEDF81E0B6
:10053000CCDFC8010197F1F786E0C7DF1F910F916B
:100540000895CF93DF93EC0102C02196C4DF888128
:100550008823D9F7DF91CF910895CF93DF93EC01F2
:1005600004C0FE0184912196B6DF88818823C9F7F3
:10057000DF91CF9108950F931F93CF93DF938C0159
:10058000862F90E08770907023E0880F991F2A953E
:10059000E1F780649ADFC0E0D0E0F801EC0FFD1FC6
:1005A000E4918E2F98DF2196C830D105B1F7DF9105
:1005B000CF911F910F910895991B79E004C0991F65
:1005C000961708F0961B881F7A95C9F780950895AD
:1005D000AA1BBB1B51E107C0AA1FBB1FA617B70769
:1005E00010F0A61BB70B881F991F5A95A9F7809585
:0C05F0009095BC01CD010895F894FFCF58
:1005FC004C696D3A005E5E5E5E5E5E5E5E00202063
:10060C00202020202020002043002020202020001B
:00000001FF
